:020000020000FC
:0200000029C015
:0200040045C1F4
:02003400D4C036
:10005400FF2408E00EBF0FE50DBFA39A8C9A8D9A7A
:100064008E9A8F9A332705B70D7F016005BF0BB7B2
:100074000F7500640BBF549A539A579A06E800BD53
:10008400002700BD09E109B9789420D415D5DFD53E
:1000940080D37DD400916000A5D37BD378D4109114
:1000A40060000117C9F400E00093600003E30093CB
:1000B400610002E20093620007E00093630001E044
:1000C4000093640001E00093650002E10093660080
:1000D40000E10093670025D46FD28DE0FBD083E567
:1000E400F9D08EE4F7D08AE3F5D080E2F3D080D261
:1000F40080E2F0D080E2EED084E4ECD083E5EAD074
:1001040081E3E8D088E3E6D000917B00083219F05F
:1001140083E5E0D002C082E4DDD082E3DBD080E37B
:10012400D9D080E2D7D080E2D5D080E2D3D05AD3E0
:1001340026D50BD184E4DED02AE093D500E3040F66
:10014400003311F400E20BC00A3311F40AE207C0D1
:100154000B3311F400E303C00C3309F403E28FE81A
:10016400D4D4802FE9D4802FB5D02ED32A9529F763
:100174008DE0B0D00CD44AD480E2ACD080E2AAD0D6
:1001840080E2A8D080E8C1D4E8E6F0E02EE08191D6
:10019400D3D42A95E1F780ECB8D4ECECF0E0E9D4C0
:1001A400EAE4FCE0E0D4D1D08827EBD0882755D10D
:1001B400882769D287E48ED082E78CD081E68AD002
:1001C40084E688D080E286D083E484D080E282D042
:1001D40080E280D080E27ED0ACCF0F930FB70F9334
:1001E4001F932F93BF93AF930CB1043509F046C00E
:1001F4005F9BFECF0CB1003209F040C05F9BFECF85
:100204000CB1005302955F9BFECF1CB11053010F3C
:10021400009364005F9BFECF0CB1005302955F9B7B
:10022400FECF1CB11053010F009365005F9BFECFFE
:100234000CB1005302955F9BFECF1CB11053010F0C
:10024400009366005F9BFECF0CB1005302955F9B49
:10025400FECF1CB11053010F009362005F9BFECFD1
:100264000CB1005302955F9BFECF1CB11053010FDC
:100274000093610000270093600053D3AF91BF91B6
:100284002F911F910F910FBF0F9118950F930FB7D7
:100294000F931F93EF93FF939B9B02C0AB980FC0E8
:1002A400AB9AECEAFCE0E30FFF1D049110B3102BB2
:1002B4000F60102312BB3395343009F433277BD2FB
:1002C40010B31F7012BBFF91EF911F910F910FBFDD
:1002D4000F9118955D9BFECF8CB90895A29AAA98A8
:1002E4004FD2AA9AA2983AD230D22FD29A99F6CF64
:1002F4003ED208951F93A29A18E0879528F0AA98F1
:1003040036D2AA9A22D204C0AA981FD2AA9A2FD26D
:100314001A9599F71F9108951F9318E0A29AAA9825
:1003240001D200D2AA9AA29810D29A9902C0E89453
:1003340001C068941CD21EF08894879502C008946A
:1003440087951A9559F71F910895C8DF85E5D2DF7F
:1003540080917B00CFDF80917C00CCDF80917D0099
:10036400C9DF80917E00C6DF80917F00C3DF80916A
:100374008000C0DF80918100BDDF80918200BADF00
:1003840008950F932F93AF93BF9309E0809FA3E841
:10039400B0E0A00DB11D8EEBADDF29E0BDDF8D9384
:1003A4002A95E1F7BF91AF912F910F910895CDDF79
:1003B40084E4A0DF17D2C9DF8827E3DF88274DD084
:1003C400882761D108950F931F932F93AF93BF9301
:1003D400EF93FF93982F112708E0109FE8EDF6E0C4
:1003E400E00DF11DABE7B0E028E005910D932A95EF
:1003F400E1F7ABDF84E47EDF13959A9569F7FF910B
:10040400EF91BF91AF912F911F910F9108950F9389
:100414001F932F93AF93BF93EF93FF93982F1127BD
:1004240008E0109FE8EDF6E0E00DF11DABE7B0E069
:1004340028E005910D932A95E1F787DF812FA1DF4D
:10044400812F0BD013959A9559F7FF91EF91BF9196
:10045400AF912F911F910F9108950F931F939F9325
:10046400EF93FF93CF93DF9309E0809FE3E8F0E0FD
:10047400E00DF11D07E0809FCBECD0E0C00DD11D55
:1004840000917B00083209F449C000E3088301812C
:100494000F3F31F40DE2088300810095039500833A
:1004A4000080069404E6009E802D912D49970681D4
:1004B40010E1101B04E6109F10E1212EFAD0012D4B
:1004C400083008F00394800D9F1D10E3082E192EA8
:1004D40004E6202EEED0812D112404E6202EE9D04E
:1004E40008810D3211F0010E0882012C11240AE05A
:1004F400202EDFD0010E0982110E1A820CE20B832A
:10050400082E11240AE0202ED4D0010E0C82110EE4
:100514001D8200E20E8300270F8346C000E3088398
:100524000181087F083F31F40DE2088300810095C2
:10053400039500830181063009F01CF400340CF4A7
:1005440002C011E3188302951081107F1295010FE8
:100554001124002E04E6202EACD0012C11240AE034
:10056400202EA7D010E3010E0982110E1A820CE28C
:100574000B8300810F7015E0019F002D1DE7019F83
:1005840004E6202E96D0002D023308F003941124A3
:100594000AE0202E8ED010E3010E0C82110E1D8273
:1005A40000E20E8300270F83DF91CF91FF91EF913B
:1005B4009F911F910F91089591DE83E39BDEACDE42
:1005C40080937B00A9DE80937C00A6DE80937D006F
:1005D400A3DE80937E00A0DE80937F009DDE809367
:1005E40080009ADE8093810097DE809382000895D4
:1005F40082E270DE80917B0018D080917C0015D05F
:1006040080917D0012D080917E000FD080917F0078
:100614000CD08091800009D08091810006D0809117
:10062400820003D082E256DE08950F931F9300E305
:1006340017E3982F807F82958A3014F4800F01C0CD
:10064400810F48DE892F8F708A3014F4800F01C027
:10065400810F40DE80E23EDE1F910F9108950F93DB
:100664002F93AF93BF9309E0809FA3E8B0E0A00D60
:10067400B11D29E08D912EDE2A95E1F7BF91AF914E
:100684002F910F9108950F932F938F93AF93BF934F
:1006940007E0809FABECB0E0A00DB11D27E08D9189
:1006A40019DE2A95E1F7BF91AF918F912F910F91A8
:1006B40008950F930FB70F9308E0000C111C10F06E
:1006C400121410F0121803940A95B9F70F910FBF82
:1006D4000F91089510E0AFED01080087108FD7ED5A
:1006E4000108003310F9A4ED0108003A1025F0EDDB
:1006F4000108000910EAB7ED0108000A10B5ECED95
:10070400010800E51012A3ED010800BA10EAB7EDE4
:100714000108000A10B5ECED010800E51012A3ED84
:10072400010800BA00000000000000000000000002
:1007340000000000000008958F939F9380E190E0F3
:100744000197F1F79F918F9108958F939F9384E27E
:1007540090E00197F1F79F918F9108958F939F9364
:1007640084EC90E0019739F49F918F9108958F93D1
:100774009F938CE891E00197F1F79F918F910895F1
:100784008F939F938CEC97E00197F1F79F918F9152
:1007940008958F939F938CE99FE00197F1F79F91C0
:1007A4008F9108958F939F938CE19EE40197F1F7C5
:1007B4009F918F9108958F939F938CE39CE9019768
:1007C400F1F79F918F910895AF93AAE0F4DFAA9572
:1007D400E9F7AF910895AF93A2E3EDDFAA95E9F7A6
:1007E400AF910895AF93A4E6E6DFAA95E9F7AF9138
:1007F4000895AF93BF93A4EFB1E0DDDF1197E9F75C
:10080400BF91AF910895AF93BF93A8EEB3E0D3DF48
:100814001197E9F7BF91AF910895AF93BF93A0E704
:10082400B7E1C9DF1197E9F7BF91AF910895AF938D
:10083400BF93A0E6BAEEBFDF1197E9F7BF91AF917E
:100844000895AF93BF936EDF1197E9F7BF91AF910E
:100854000895AF93BF9379DF1197E9F7BF91AF91F3
:100864000895AF93BF9383DF1197E9F7BF91AF91D9
:100874000895AA2319F4BB2309F40895AF93BF93F1
:1008840088DF1197E9F7BF91AF910895AF93BF93B4
:1008940092DF1197E9F7BF91AF910895AF93BF939A
:1008A40093DF1197E9F7BF91AF910895AF93BF9389
:1008B40099DF1197E9F7BF91AF910895AF93BF9373
:1008C400ACDF1197E9F7BF91AF910895882781B9FB
:1008D4008CE080B9089584EA86BF86B787FFFDCF90
:1008E40091B1987F089583B984E886BF86B787FF5E
:1008F400FDCF91B1987F089584EC86BF86B787FFBA
:10090400FDCF83B191B1987F089584E886BF86B7FF
:1009140087FFFDCF83B191B1987F089584E986BFA5
:100924000895D9DF983089F580EDDDDF983169F5D8
:1009340080E0D9DF983249F580916000D4DF9832A5
:1009440021F580916100CFDF9832F9F48091620043
:10095400CADF9832D1F480916300C5DF9832A9F4DC
:1009640080916400C0DF983281F480916500BBDF20
:10097400983259F480916600B6DF983231F4809150
:100984006700B1DF983209F400C0C8DF0895A3DF1F
:10099400983011F09031C1F580EDA5DF9831A1F5C3
:1009A40080E0A1DF983281F596DF903169F581ED21
:1009B4009ADF903449F5A0DF80936000903521F5EB
:1009C4009BDF809361009035F9F496DF8093620099
:1009D4009035D1F491DF809363009035A9F48CDFD6
:1009E40080936400903581F487DF809365009035AF
:1009F40059F482DF80936600903531F486DF80936A
:100A04006700983509F400C089DF08958091640077
:100A140043D090936800809369008EE280936A00CB
:100A240059DC8091650038D090936B0080936C0002
:100A34008EE280936D004EDC809166002DD0909301
:100A44006E0080936F0080E28093700043DC80919D
:100A5400620022D090937100809372008AE38093A5
:100A6400730038DC8091610017D0909374008093F8
:100A740075008AE3809376002DDC809160000CD0B1
:100A8400909377008093780080E28093790022DC51
:100A9400882780937A0008950F931F9300E3182FFB
:100AA400807F8295800F16DC982F812F8F70800FA6
:100AB40011DC1F910F9108950F9307B30C6F07BBBF
:100AC40083DE08B30063037308BB1AD06BDE08B37C
:100AD4000063037308BB14D008B30063037308BB3B
:100AE4000FD008B30062037208BB0AD088E20DD0AD
:100AF4008FE00BD086E009D08CE007D00F910895E9
:100B0400C39A35DEC3983CDE08950F931F93082FD4
:100B1400007F18B3102B0F6010231B7F18BBF0DF6E
:100B24008F70829518B3182B8F6018231B7F18BB06
:100B3400E7DF1F910F9108950F931F93082F007FF4
:100B440018B3102B0F601023146018BBD9DF8F70FB
:100B5400829518B3182B8F601823146018BBD0DF4C
:100B64001F910F9108958591803011F0E5DFFBCF3F
:100B740008958191803011F0DFDFFBCF089581E08B
:100B8400C4DF10DE08950F93880F880F880FE82FB5
:100B9400F5E0FF1F8064B9DF08E0C895802DCCDF45
:100BA40031960A95D1F70F91089504041F040400A7
:100BB4001F000C0204080E0000000C020C020C00C2
:100BC40000001806010618001F00030C100C030097
:100BD4001F0004041F041F040400001F001F001F43
:100BE400000015151515151515002020203A202094
:100BF400202020202F20202F2020000070706D2026
:100C040000000020012002200320042005200620EB
:100C140007202020446973706C61792D54657374C6
:100C240020004368617220362D3820626C696E6B37
:100C3400656E0000437572736F722D506F732E20B2
:100C44003D203635000047726164204300000F9355
:100C54000AB30867087F0ABB0BB307600BBB0F918D
:100C640008950F9300274CE0DB9ADC9ADD9ADE9816
:100C7400CA9B13C04A95C99B10C04A95C89B0DC016
:100C84004A95CD9B02C0DD98F3CFCC9B02C0DC9883
:100C9400EFCFCB9B07C0DB98EBCF002319F079DDB6
:0C0CA4000A95E1CF0F9108955060A090D8
:00000001FF
